:1000000018308A0000280000FF00030E8301A100C1
:100010000A08A0008A010408A2007708A300780853
:10002000A4007908A5007A08A600831383128C30F7
:100030008400001C1D280C1832288B1E21280B1947
:100040003528220884002308F7002408F800250832
:10005000F9002608FA0020088A00210E8300FF0E0E
:100060007F0E09008A110A1223298A110A12912986
:100070008E30F70083164308F8004208F900FA01B1
:10008000F808031D4D287908F800F9010830F70237
:10009000F808031D4D28F70155280310F81B5428B4
:1000A000F90DF80DF7034D28F81383120800831695
:1000B000420803191D29CE00460803191D29CE0246
:1000C000031C67287F30CE0703181D296D28813057
:1000D000CE02031C1D2903191D294E08F700F80143
:1000E000F901FA01CD014308CC00CC174408CB003C
:1000F0004508CA001930CE004908CA0203189028E2
:100100000130CB0203189028CC0203189028CD02AE
:1001100003189028CD0ACC0ACB0A4908CA07C2287E
:100120004808CB020318AB280130CC020318AB28D7
:10013000CD020318AB28CD0ACC0A4808CB074908E2
:10014000CA07031CC228CB0A031DC228CC0A031D00
:10015000C228CD0AC22847088038CC020318C1281B
:100160000130CD020318C128CD0A47088038CC07DA
:100170004808CB07031C9F28CC0A031D9F28CD0AE3
:100180009F287A14CE0BC528D0280310CA0DCB0D9A
:10019000CC0DCD0D0310FA0DF90DF80DCF0D7C2807
:1001A0004F1CD8280310F80CF90CFA0CCF0CDB28E4
:1001B000F70303191D29CF1B04290310CA0DCB0D0A
:1001C000CC0DCD0D4908CA020318F0280130CB022E
:1001D0000318F028CC020318F028CD02031C1329C1
:1001E0004808CB020318FB280130CC020318FB2877
:1001F000CD02031C132947088038CC0203180429B8
:100200000130CD02031C1329FA0A031D1329F90A30
:10021000031D1329F80A031D1329F70A03191D29C1
:10022000F80CF90CFA0C4308CE004708CE06CE1F96
:100230001B29F8172129F8132129F701F801F901E1
:10024000FA018312080030088316C10083122F08B8
:100250008316C000C301FF30C2001030C400F70194
:10026000FA01C10CC00C031C3B294208F707031814
:10027000FA0A4308FA07FA0CF70CF90CF80CC40B4D
:1002800031297908C1007808C0008312010883165B
:10029000C0070318C10A4108C3004008C200831206
:1002A00038207A088316C5007908C4007808C3008E
:1002B0007708C2008030C900C801C7017E30C6007F
:1002C000831257207A08B4007908B3007808B20086
:1002D0007708B10034088316C500831233088316EB
:1002E000C400831232088316C300831231088316B8
:1002F000C200C901C801C7018030C600831257205F
:100300007A08B4007908B3007808B2007708B10021
:10031000B001AF0181018F018E010C108A110A1208
:100320002128AF0A0319B00A0B118A110A122128D9
:100330000D050D052310CD32F4326F396F36EF33D2
:10034000E931EB30A039F430EE34E332A01273100F
:10035000A82129103218B119A03BF73BAE36EC307A
:100360006217633DA0060A00301731000D05231007
:10037000C13AF437721DA0127310D037733665324C
:10038000EE34A03A7039613B611DA01273100D0567
:100390000001CA306E104334F237F5397400B11AD7
:1003A0002E1A2E19B01833002310F6327210F037BF
:1003B000F230E434200061346C34743469346D34C8
:1003C000653474345F3474345B34B03443345D3436
:1003D000203461346C34743469346D34653474346D
:1003E0005F3461345B346D345D34203461346C349B
:1003F000743469346D34653474345F3470345B3410
:10040000503461345D3420340034733468347434CF
:100410005F3474345B34B03443345D34203473342B
:10042000683474345F3468345B34253425345D3487
:100430002034203441346E3465346D346F345B3491
:100440006D342F3473345D3463346834653463340D
:100450006B340D340A340D340A3400340830F8009B
:1004600000008711A8112808831687000000F30DEB
:1004700083120712031C422A2816280883168700B5
:10048000462A831228122808831687000000831248
:10049000A8152808831687008312871D4D2AF80B9C
:1004A000302A00008711A811280883168700000051
:1004B0008312281628088316870000000000831284
:1004C000A8152808831687008312871D652AF8015E
:1004D0000000071A78148711A811280883168700CE
:1004E0008312071228122808831687008312080037
:1004F000281628088316870000008312A8152808EC
:10050000831687000000831207122812280883161A
:100510008700000083128711A8112808831687001E
:100520008030F30083122E22FE30F3002E22281298
:1005300028088316870000008312A8152808831650
:1005400087008312871DA22A0000A62A0000281611
:10055000280883168700000083128A150A1692283D
:100560000830F4007708F50028162808831687005D
:1005700000008312A8152808831687008312871DA0
:10058000BF2A071A0314071E0310F80D0000A81154
:1005900028088316870083128711F40BB42A2816C3
:1005A00028088316870000008312071275080319B4
:1005B000DE2A281228088316870083120000A81557
:1005C0002808831687008312871DE42A00008711FC
:1005D000A81128088316870000008312071228122A
:1005E000280883168700831208006530840083136F
:1005F00000080319082B0230F800F701F70BFE2A58
:10060000F80BFD2A9730F700F70B042B800BFB2A21
:100610000800281628088316870000008312A815F2
:100620002808831687000000831207122812280862
:1006300083168700000083128711A81128088316EB
:1006400087008030F30083122E22E730F3002E2241
:10065000281628088316870000008312A81528088A
:100660008316870000008312871D342B071228127F
:10067000280883168700000083128711A811280814
:10068000831687008130F30083122E22F701B022F7
:100690007808E10061083A396004E100281628086A
:1006A0008316870000008312A81528088316870088
:1006B00000008312871D5A2B071228122808831660
:1006C0008700000083128711A8112808831687006D
:1006D0008030F30083122E22E630F3002E226108D0
:1006E000F3002E22281228088316870000008312A8
:1006F000A8152808831687008312871D7D2B00000C
:10070000812B0000281628088316870000000A3075
:100710008312E500F52228162808831687000000BA
:100720008312A81528088316870000008312071279
:100730002812280883168700000083128711A81149
:100740002808831687008030F30083122E22E730BA
:10075000F3002E2228162808831687000000831233
:10076000A81528088316870000008312871DB62B62
:1007700007122812280883168700000083128711A9
:10078000A8112808831687008130F30083122E22D7
:10079000F701B0227808E1006108F8008A150A160E
:1007A0009A28A81328088316870083128713083015
:1007B000F800DA2B0000F817EB2BF813E40C031801
:1007C0008717031C87137817EB2B7813F80BDE2B96
:1007D000E92B000087173F308400840BED2B0000CD
:1007E000F81BDD2B781BE52B0800831603178C17ED
:1007F0000C14000000000318242C83120C087F390D
:100800000313E10003170D080313E20003170F0899
:100810000313E3006108E400D123620803178D008D
:100820000313630803178F0083168C170C14000042
:10083000000083120313E00B1E2C212C83160317D8
:10084000242C432C8316031783120C0D0E0D7F39B5
:100850000313E10003170D080313E20003170F0849
:100860000313E3006108E400D123620803178D003D
:100870000313630803178F008D0A03198F0A0310EF
:100880000313E00BF52B0800831603178C170C14C9
:100890000000000083120C087F390319882C031311
:1008A000E00003170D080313E10003170F080313FB
:1008B000E2006008E400D123610803178D000313F0
:1008C000620803178F0083168C170C1400000000B9
:1008D00083120C0D0E0D7F390319882C0313E000D1
:1008E00003170D080313E10003170F080313E200B9
:1008F0006008E400D123610803178D000313620828
:1009000003178F008D0A03198F0A0313442C031752
:1009100003130800831603178C170C140000000043
:1009200083120D080313E10003170F080313E200FD
:1009300003170C080313E400D123610803178D008B
:100940000313620803178F008D0A03198F0A03131C
:10095000E00B8A2C0800983003178D0001308F00BF
:1009600003101D300313E000F523B43003178D008E
:1009700001308F0003134424A73003178D0001308A
:100980008F00031418300313E000F523B63003176B
:100990008D0001308F0003100B300313E000F523AE
:1009A000C93003178D0001308F0003134424BC307D
:1009B00003178D0001308F00031412300313E00081
:1009C000F523CF3003178D0001308F00031344242B
:1009D0002030E400D1230D30E400D1230A30E400BC
:1009E000D123D43003178D0001308F00031344242A
:1009F000DB3003178D0001308F0083168C170C1429
:100A00000000000083128C0803191D2D0D0803132C
:100A1000E00003170F080313E10003170C0803138A
:100A2000E400D123600803178D0003136108031746
:100A30008F008D0A03198F0AFD2C05308D000230BE
:100A40008F0010300313E0008A242530E400D12306
:100A5000173003178D0002308F0016300313E000AB
:100A60008A248A150A16A6282816280883168700BD
:100A700000008312A815280883168700000083123F
:100A80000712281228088316870000008312871196
:100A9000A8112808831687003C30F30083122E2209
:100AA000F3012E227030F3002E222812280883161C
:100AB000870000008312A815280883168700831278
:100AC000871D602D0000642D00002816280883165D
:100AD0008700000006308312E500F522281628085A
:100AE0008316870000008312A81528088316870044
:100AF00000008312071228122808831687000000BE
:100B000083128711A8112808831687003C30F30050
:100B100083122E220130F3002E22E030F3002E2229
:100B2000281228088316870000008312A8152808B9
:100B3000831687008312871D9B2D00009F2D0000C8
:100B40002816280883168700000006308312E50067
:100B5000F522281628088316870000008312A8159E
:100B6000280883168700000083120712281228081D
:100B700083168700000083128711A81128088316A6
:100B800087003C30F30083122E220230F3002E2225
:100B9000F3012E22281228088316870000008312F2
:100BA000A8152808831687008312871DD52D0000FD
:100BB000D92D00002816280883168700000006306B
:100BC0008312E500F5228A150A16AB282816280894
:100BD0008316870000008312A81528088316870053
:100BE00000008312071228122808831687000000CD
:100BF00083128711A811280883168700C030F300DC
:100C000083122E222630F3002E22B830F3002E223B
:100C1000281228088316870000008312A8152808C8
:100C2000831687008312871D132E0000172E0000E5
:100C30002816280883168700000083122816280823
:100C40008316870000008312A815280883168700E2
:100C5000000083120712281228088316870000005C
:100C600083128711A811280883168700C030F3006B
:100C700083122E221330F3002E220730F3002E228F
:100C8000281228088316870000008312A815280858
:100C9000831687008312871D4B2E00004F2E000005
:100CA00028162808831687000000831228162808B3
:100CB0008316870000008312A81528088316870072
:100CC00000008312071228122808831687000000EC
:100CD00083128711A811280883168700C030F300FB
:100CE00083122E222630F3002E223930F3002E22DA
:100CF000281228088316870000008312A8152808E8
:100D0000831687008312871D832E0000872E000024
:100D10002816280883168700000083128A150A16F1
:100D2000BB28281628088316870000008312A81500
:100D3000280883168700000083120712281228084B
:100D400083168700000083128711A81128088316D4
:100D50008700C030F30083122E227008F3002E2289
:100D6000281628088316870000008312A815280873
:100D70008316870000008312871DBC2E07122812DD
:100D8000280883168700000083128711A8112808FD
:100D900083168700C130F30083122E22F701B022A0
:100DA0007808F100281228088316870000008312B3
:100DB000A8152808831687008312871DDD2E0000E2
:100DC000E12E00002816280883168700000071080D
:100DD000F800831208000430F00091267808E00043
:100DE0000530F0009126780EF7000F30F7057708F0
:100DF000A7018B1BA7178B138316C301C200831295
:100E00003820A71B8B177708E9007808EA007908D3
:100E1000EB007A08EC00A7018B1BA7178B136C085B
:100E20008316C50083126B088316C40083126A08F8
:100E30008316C300831269088316C200C901C80162
:100E4000C7018330C60083125720A71B8B177A086F
:100E5000E4007908E3007808E2007708E100A701E0
:100E60008B1BA7178B138316C3018312600883168D
:100E7000C20083123820A71B8B1783107A088316B1
:100E8000AC007908AB007808AA007708A9008312A3
:100E900064088316B000831263088316AF008312C0
:100EA00062088316AE00831261088316AD008A15AE
:100EB000831200208A117A08E8007908E700780890
:100EC000E6007708E5006508F7006608F80067089F
:100ED000F9006808FA008A150A16CB288316290833
:100EE0000319DF2FB1002D080319DF2FB1070318F5
:100EF000802F7F30B102031CDF2F0319DF2F842FD7
:100F00008130B1070318DF2F3108F700F801F9012C
:100F1000FA012A08B500B5172B08B4002C08B30055
:100F20001830B100B201331CAD2F3008FA07031C92
:100F30009F2FF90A031D9F2FF80A0319B2172F08D4
:100F4000F907031CA62FF80A0319B2172E08AB00E5
:100F5000AB172B08F8070318B217B20DF80CF90CF1
:100F6000FA0CB50CB40CB30C0310B10B922F01307A
:100F7000F7070318DF2FF81BC42FB50DFA0DF90D75
:100F8000F80DF7030319DF2FB51FD52FFA0A031D3C
:100F9000D52FF90A031DD52FF80A031DD52FF80CFC
:100FA000F90CFA0CF70A0319DF2F2A08B2002E08F1
:100FB000B206B21FDD2FF817E32FF813E32FF70166
:100FC000F801F901FA0183120800FC017208FB0024
:100FD000FC00FB0173087B07F4007C08F500031894
:0C0FE000F50A7408F8007508F900080014
:101000008030831C06288316AE0683128316B30134
:10101000B4012A08B2002E08B20629080319F428E0
:10102000B100F7002D080319FD28B1020319992812
:10103000031C57282E08B700B7172F08B600300832
:10104000B500B4010310B70CB60CB50CB40CB10B61
:101050002128B21F2E2833141129331031103316D2
:10106000AC308400831326293312B21B4128311C73
:101070004C28B70CB60CB50CB40CF70A03190C29A4
:101080004C28B71B4F280310B40DB50DB60DB70D86
:10109000F70303190C2941283317B92833132A08F9
:1010A000B200B21F5528B7170529B71305292D0817
:1010B000B100F7002908B1022A08B700B7172B08BA
:1010C000B6002C08B500B4010310B70CB60CB50C73
:1010D000B40CB10B6328B21F7028B3141129B310DC
:1010E0003110B316B030840083132629B312B21B1B
:1010F0008328311C8E28B70CB60CB50CB40CF70A3B
:1011000003190C298E28B71B91280310B40DB50DB7
:10111000B60DB70DF70303190C298328B317B928A7
:10112000B3132E08B200B21F9728B7170529B713BB
:1011300005292E08B700B7172F08B6003008B500EC
:10114000B21FA628B713331511293311B40131107A
:10115000AC30840083132629B21BCF282A08B200A2
:10116000311CB928B70CB60CB50CB40CF70A03192E
:101170000C29B41FCA28B50A031DCA28B60A031DC4
:10118000CA28B70A031DCA28B70CB60CB50CF70A53
:1011900003190C29331B4E28B31B9028EE288030EE
:1011A000B706B71FD72811292E08B200E4282A084D
:1011B000B200B708031DE428B608031DE428B508EB
:1011C000031DE428F7010529B71BEE280310B40D11
:1011D000B50DB60DB70DF70BE4280C29B21FF22898
:1011E000B7170529B71305292D08F7002E08B700F2
:1011F0002F08B6003008B50005292908F7002A088D
:10120000B7002B08B6002C08B5003708F8003608E0
:10121000F9003508FA004429F701F801F901FA014B
:101220004429B401B509B609B709B409B40A031DC4
:101230001F29B50A031D1F29B60A0319B70A331857
:101240002D28B3186F283319A528D4280008B5070E
:10125000031C3029B60A031D3029B70A03193114BB
:1012600084030008B607031C3829B70A0319311490
:1012700084030008801F803AB70703183114331A1B
:101280003428B31A7628AC28831208000130F00005
:101290008A1191268A15E301E201E1017808E00054
:1012A0000230F0008A1191268A15E5017808E400E1
:1012B0000330F0008A1191268A157808E600660D41
:1012C000E700E70DFC30E705660EF700F70CF70CBA
:1012D0000330F7057708A7018B1BA7178B1383161D
:1012E000C301C2008A11831238208A15A71B8B17ED
:1012F0007708F1007808F2007908F3007A08F40022
:10130000A7018B1BA7178B1374088316C5007308DE
:10131000C4007208C3007108C200C901C801C70136
:101320008130C6008A11831257208A15A71B8B179C
:101330007A08EF007908EE007808ED007708EC00F5
:10134000F101600DF200610DF300620DF400F20D89
:10135000F30DF40DFC30F205640DF900650DFA0093
:10136000F90DFA0DFC30F9057908F1047A08F20458
:10137000660EF700F70CF70C0330F70577087104D9
:10138000F7007208F8007308F9007408FA007A0888
:10139000FE007908FD007808FC007708FB00B630F5
:1013A000F700FA01F901F8017B087C047D047E0452
:1013B000031DDC29F701E9290310F81BE829FB0DBF
:1013C000FC0DFD0DFE0DFA0DF90DF80DF70BDC29E6
:1013D000F8137708F1007808F2007908F3007A082A
:1013E000F400831074088316AC007308AB00720815
:1013F000AA007108A90083126F088316B000831237
:101400006E088316AF0083126D088316AE00831238
:101410006C088316AD00831200207A08EB0079086F
:10142000EA007808E9007708E8006808F70069082A
:10143000F8006A08F9006B08FA008A150A16D7281E
:10144000281628088316870000008312A81528088C
:1014500083168700000083120712281228088316BB
:101460008700000083128711A811280883168700BF
:10147000C030F3008A1183122E228A152630F30021
:101480008A112E228A15B830F3008A112E228A156D
:10149000281228088316870000008312A815280840
:1014A000831687008312871D532A0000572A0000E5
:1014B000281628088316870000008312281628089B
:1014C0008316870000008312A8152808831687005A
:1014D00000008312071228122808831687000000D4
:1014E00083128711A811280883168700C030F300E3
:1014F0008A1183122E228A151330F3008A112E22AC
:101500008A150730F3008A112E228A15281228081E
:101510008316870000008312A81528088316870009
:101520008312871D912A0000952A0000281628089A
:101530008316870000008312281628088316870068
:1015400000008312A8152808831687000000831264
:1015500007122812280883168700000083128711BB
:10156000A811280883168700C030F3008A1183125F
:101570002E228A152630F3008A112E228A15B930C0
:10158000F3008A112E228A15281228088316870054
:1015900000008312A8152808831687008312871D70
:1015A000CF2A0000D32A00002816280883168700B7
:1015B000000083128A150A16E2280130F0008A1111
:1015C00091268A15E1017808E0000230F0008A11C6
:1015D00091268A157808E2000330F0008A119126DE
:1015E0008A15780EF7000F30F7057708A7018B1BD7
:1015F000A7178B138316C301C2008A1183123820E8
:101600008A15A71B8B177708EB007808EC00790880
:10161000ED007A08EE00A7018B1BA7178B137A0841
:101620008316C500831279088316C40083127808D4
:101630008316C300831277088316C200C901C8014C
:10164000C7018330C6008A11831257208A15A71B51
:101650008B177A08E6007908E5007808E400770837
:10166000E3006008ED00EC016C086204F70060081C
:10167000FA007708A7018B1BA7178B138316C200EC
:101680007A08C3008A11831238208A15A71B8B178A
:101690007708EC007808ED007908EE007A08EF0092
:1016A00083107A088316AC00831279088316AB0086
:1016B000831278088316AA00831277088316A9007C
:1016C000831266088316B000831265088316AF0084
:1016D000831264088316AE00831263088316AD007C
:1016E000831200207A08EA007908E9007808E80007
:1016F0007708E7006708F7006808F8006908F9004C
:101700006A08FA008A150A16F0282816280883168F
:10171000870000008312A8152808831687000000A0
:101720008312871D912B0712281228088316870021
:10173000000083128711A8112808831687008030C3
:10174000F3008A1183122E228A15E330F3008A11E6
:101750002E228A152812280883168700000083127B
:10176000A8152808831687008312871DB52B000053
:10177000B92B000028162808831687000000643063
:101780008312E5008A11F5228A1528162808831687
:10179000870000008312A815280883168700000020
:1017A000831207122812280883168700000083126C
:1017B0008711A8112808831687008130F3008A1149
:1017C00083122E228A150130F7008A11B0228A1561
:1017D0007808E0000130F7008A11B0228A157808F5
:1017E000E100F7018A11B0228A157808E200281278
:1017F00028088316870000008312A815280883167E
:1018000087008312871D022C0000062C000028167A
:1018100028088316870000008312E10CE10C3F309A
:10182000E105E6016008E500E600E501610EF7006C
:10183000F030F70577086507E3006608E400031851
:10184000E40AA7018B1BA7178B1364088316C30038
:10185000831263088316C2008A11831238208A1506
:10186000A71B8B177708E5007808E6007908E700E2
:101870007A08E800A7018B1BA7178B13680883164B
:10188000C500831267088316C40083126608831696
:10189000C300831265088316C200C901FF30C80067
:1018A0007F30C7008E30C6008A11831257208A15F8
:1018B000A71B8B1752308316AC00B830AB002F300B
:1018C000AA008630A9007A08B0007908AF0078082D
:1018D000AE007708AD008A1183126E278A15831037
:1018E00066308316AC00AB00BB30AA008430A90080
:1018F0007A08B0007908AF007808AE007708AD002C
:10190000831200208A150A16FB2828162808831639
:10191000870000008312A81528088316870000009E
:1019200083120712281228088316870000008312EA
:101930008711A8112808831687008030F3008A11C8
:1019400083122E228A15E530F3008A112E228A1581
:101950006430E5008A11F5228A15281628088316B6
:10196000870000008312A81528088316870000004E
:101970008312871DB92C07122812280883168700A6
:10198000000083128711A811280883168700813070
:10199000F3008A1183122E228A150130F7008A1172
:1019A000B0228A157808E0000130F7008A11B022D1
:1019B0008A157808E100F7018A11B0228A157808A3
:1019C000E200281228088316870000008312A81559
:1019D0002808831687008312871DEC2C0000F02C4A
:1019E0000000281628088316870000008312E10CE7
:1019F000E10C3F30E105E6016008E500E600E501A5
:101A0000610EF700F030F70577086507E300660818
:101A1000E4000318E40AA7018B1BA7178B136408C3
:101A20008316C300831263088316C2008A118312CF
:101A300038208A15A71B8B177708E5007808E60081
:101A40007908E7007A08E800A7018B1BA7178B131A
:101A50007A088316C500831279088316C40083129E
:101A600078088316C300831277088316C200C90161
:101A7000FF30C8007F30C7008E30C6008A11831245
:101A800057208A15A71B8B178316AC01AB017A3040
:101A9000AA008530A9007A08B0007908AF0078085C
:101AA000AE007708AD008A1183126E278A15831065
:101AB0008316AC01AB01C030AA008130A9007A08BE
:101AC000B0007908AF007808AE007708AD00831247
:101AD00000208A150A16062928162808831687006A
:101AE00000008312A81528088316870000008312BF
:101AF0000712281228088316870000008312871116
:101B0000A8112808831687003C30F3008A1183123D
:101B10002E228A157208F3008A112E228A152812A5
:101B200028088316870000008312A815280883164A
:101B300087008312871D9A2D00009E2D0000281615
:101B400028088316870000008312281628088316A9
:101B5000870000008312A81528088316870000005C
:101B600083120712281228088316870000008312A8
:101B70008711A8112808831687003D30F3008A11C9
:101B800083122E228A15F7018A11B0228A1578084D
:101B9000F2007208F80008008E30F7007308F800B1
:101BA0007208F900FA01F31FDA2DF809F909F90AA8
:101BB0000319F80AF808031DE72D7908F800F90160
:101BC0000830F702F808031DE72DF701F02D031088
:101BD000F81BEE2DF90DF80DF703E72DF31FF813A1
:101BE000080083162608AD002A08AD06AD1FFD2D9E
:101BF00003110310A61B0314302E2608AD0029087C
:101C0000AE002508AE0203190B2EAD1F302E0308BF
:101C1000013A8300302E2A08AE002608AE020319CE
:101C2000172EAD1F302E0308013A8300302E2B08EB
:101C3000AE002708AE020319232EAD1F302E030875
:101C4000013A8300302E2C08AE002808AE0203199A
:101C50002F2EAD1F302E0308013A8300302E0310C3
:101C600083120800350884008313361883176D0823
:101C70008000840A8001B50A0319B60A08008008AA
:101C80000319542EE1010408E0006110831B611464
:101C90000008ED0032266008840083136118831762
:101CA000840A0319850A3F2E8A150A164029E8017D
:101CB0000408E7006810831B6814610EF038E30025
:101CC000E307E23EE400323EE60061080F39E40734
:101CD000E407E607E93EE500E507E507600E0F3992
:101CE000E507E607E50DE60DE609E60D60080F39A4
:101CF000E607E30D0730E2000A30E607E503031CC0
:101D00007D2EE507E403031C812EE407E303031C97
:101D1000852EE307E203031C892E623084008313BF
:101D200007306705671384076630040203196717D5
:101D30000008F700031DA42E671BA42E671AB62EF9
:101D4000E719A42E2030A72EE71567123030F707C9
:101D5000E1010408E0006110831B61147708ED00C5
:101D6000322660088400831361188317840A671F72
:101D7000942E8A150A167229F701F801F901FA0161
:101D80008316A001A101A201A301740873047204C7
:101D900071040319FD2E2030A40003108312ED0DF1
:101DA000EE0DEF0DF00D8316A00DA10DA20DA30DEC
:101DB00074082302031DE62E73082202031DE62E7B
:101DC00072082102031DE62E71082002031CF72E63
:101DD0007108A0027208031C720FA1027308031C91
:101DE000730FA2027408031C740FA3020314F70DEF
:101DF000F80DF90DFA0DA40BCD2EA030840083133D
:101E0000831208000408E5006408E70003192B2F7B
:101E100063088316AC00831262088316AB0083123A
:101E200061088316AA00831260088316A900B00116
:101E3000AF012030AE008230AD008A1183126E27D0
:101E40008A157A08E3007908E2007808E10077084B
:101E5000E000E70B082F6308F0006208EF0061085C
:101E6000EE006008ED006D08B63CED00FA016E086A
:101E7000F100EE170310EE0CEF0CF00CFA0CF90C5D
:101E8000F80CF70CED0B3A2FF11F512FF709F80959
:101E9000F909FA09F70A0319F80A0319F90A0319E3
:101EA000FA0A7A08E3007908E2007808E100770886
:101EB000E000E31F682FE503E516E009E109E20908
:101EC000E309E00A0319E10A0319E20A0319E30A24
:101ED0003B30EC009A30EB00CA30EA00E9010A30EE
:101EE000E70064080319E50A6308F0006208EF00E0
:101EF0006108EE006008ED006C08F4006B08F30068
:101F00006A08F2006908F100BC260008E000840AB3
:101F10000008E100840A0008E200840A0008E300E7
:101F2000FD308407F708031DA82F640A6702031910
:101F3000A82F65080319AA2F0F3967020319A22FCA
:101F40000318DA2FE51BDA2F651BAA2F2030D62FB6
:101F50002030E505E51EB82FE5126408031DE503F2
:101F60007708E5002D30ED0032266508F700E50121
:101F700064086702031DC62F7708E5002E30ED00C8
:101F800032266508F7002030E50500303030E51EC8
:101F9000D62FE5126408031DE5037708E5002D3010
:101FA000ED0032266508F700E5013030F7077708C5
:101FB000ED0032266C08F0006B08EF006A08EE00B6
:101FC0006908ED00F401F301F2010A30F100BC26CA
:101FD0007A08EC007908EB007808EA007708E90055
:061FE000E70B742F08005E
:102000000330F2000A128A156C250A168A11780824
:10201000EE000430F2000A128A156C250A168A11A5
:102020007808EF006E08F2006F08F3000A12E52747
:102030000A167908F1007808F0007008F8007108B5
:10204000F9007908E1007808E0000730F2000A1290
:102050008A156C250A168A117808EE000830F200FD
:102060000A128A156C250A168A117808EF006E0884
:10207000F2006F08F3000A12E5270A167908F1004A
:102080007808F0007008F8007108F9007908E3009A
:102090007808E2000530F2000A128A156C250A164B
:1020A0008A117808EE000630F2000A128A156C25B3
:1020B0000A168A117808EF006E08F2006F08F30024
:1020C0000A12E5270A167908F1007808F00070086E
:1020D000F8007108F9007908E5007808E400630861
:1020E000F3006208F2000A128A15CC250A168A113A
:1020F0007708EE007808EF007908F0007A08F10020
:102100006108F3006008F2000A128A15CC250A164D
:102110008A11A7018B1BA7178B1371088316C500A3
:102120007008C40083126F088316C30083126E0800
:102130008316C2007A08C9007908C8007808C70069
:102140007708C6000A12831257200A16A71B8B179E
:102150007A08E9007908E8007808E7007708E600DF
:102160006908F1006808F0006708EF006608EE00F3
:102170007610F6107108F5007008F4006F08F3008F
:102180006E08F20071088316A8007008A700831279
:102190006F088316A60083126E088316A500AC0193
:1021A000AB01AA01A9010A128A158312F1250A16A8
:1021B0008A11031CDF2876147308803AF300831613
:1021C000A801A701A6017F30A5007508AC0074081E
:1021D000AB007308AA007208A9000A128A158312BC
:1021E000F1250A168A11031C1629A7018B1BA717B4
:1021F0008B138316C501C401C3017F30C20075086B
:10220000C9007408C8007308C7007208C6000A1223
:10221000831257200A16A71B8B177A08F500790836
:10222000F4007808F3007708F200F6140A308316F9
:10223000AC008930AB003430AA007C30A9007508AE
:10224000B0007408AF007308AE007208AD000A1247
:1022500083126E270A1677088316A4007808A50053
:102260007908A6007A08A700AC002608AB0025086C
:10227000AA002408A9007508B0007408AF0073080C
:10228000AE007208AD000A1283126E270A16770894
:102290008316A4007808A5007908A6007A08A7008C
:1022A00083102708AC002608AB002508AA002408E4
:1022B000A9007C30B0007930AF003530AE008130FD
:1022C000AD000A128A15831200200A168A117A08B4
:1022D000FE007908FD007808FC007708FB007E0806
:1022E0008316AC007D08AB007C08AA007B08A9001F
:1022F0007508B0007408AF007308AE007208AD0036
:102300000A1283126E270A1677088316A40078082B
:10231000A5007908A6007A08A700AC002608AB0043
:102320002508AA002408A9007508B0007408AF00A9
:102330007308AE007208AD000A1283126E270A16E7
:1023400077088316A4007808A5007908A6007A0803
:10235000A70083102708AC002608AB002508AA00B8
:102360002408A9003F30B0000230AF003330AE0087
:102370008330AD000A128A15831200200A168A11D2
:102380007A08FE007908FD007808FC007708FB0059
:102390007E088316AC007D08AB007C08AA007B0891
:1023A000A9007508B0007408AF007308AE00720889
:1023B000AD000A1283126E270A1677088316A4004E
:1023C0007808A5007908A6007A08A700AC002608BE
:1023D000AB002508AA002408A9007508B0007408FD
:1023E000AF007308AE007208AD000A1283126E27A8
:1023F0000A1677088316A4007808A5007908A600B5
:102400007A08A70083102708AC002608AB0025082F
:10241000AA002408A9003330B0008C30AF001E3071
:10242000AE008330AD000A128A15831200200A160E
:102430008A117A08FE007908FD007808FC00770808
:10244000FB008316AC01AB01AA017F30A90075081F
:10245000B0007408AF007308AE007208AD000A1235
:1024600083126E270A1677088316A4007808A50041
:102470007908A6007A08A700AC002608AB0025085A
:10248000AA002408A9007508B0007408AF007308FA
:10249000AE007208AD000A1283126E270A16770882
:1024A0008316A4007808A5007908A6007A08A7007A
:1024B00083102708AC002608AB002508AA002408D2
:1024C000A9001B30B000E430AF003530AE008230E0
:1024D000AD000A128A15831200200A168A117A08A2
:1024E0008316A3007908A2007808A1007708A0004D
:1024F0002308AC002208AB002108AA002008A9008C
:102500007508B0007408AF007308AE007208AD0023
:102510000A1283126E270A1677088316A400780819
:10252000A5007908A6007A08A700AC002608AB0031
:102530002508AA002408A9007508B0007408AF0097
:102540007308AE007208AD000A1283126E270A16D5
:1025500077088316A4007808A5007908A6007A08F1
:10256000A70083102708AC002608AB002508AA00A6
:102570002408A900A430B000DB30AF006730AE0003
:102580008330AD000A128A15831200200A168A11C0
:102590007A088316A3007908A2007808A1007708BA
:1025A000A0002308AC002208AB002108AA002008E4
:1025B000A9007508B0007408AF007308AE00720877
:1025C000AD000A1283126E270A1677088316A4003C
:1025D0007808A5007908A6007A08A700AC002608AC
:1025E000AB002508AA002408A9007508B0007408EB
:1025F000AF007308AE007208AD000A1283126E2796
:102600000A1677088316A4007808A5007908A600A2
:102610007A08A70083102708AC002608AB0025081D
:10262000AA002408A9003330B0008C30AF001E305F
:10263000AE008330AD000A128A15831200200A16FC
:102640008A117A088316A3007908A2007808A100ED
:102650007708A0007508AC007408AB007308AA00E6
:102660007208A9007E08B0007D08AF007C08AE00AB
:102670007B08AD000A1283126E270A1677088316AC
:10268000A4007808A5007908A6007A08A70083129C
:10269000A7018B1BA7178B1383162708C5002608D5
:1026A000C4002508C3002408C2002308C90022086A
:1026B000C8002108C7002008C6000A12831257204C
:1026C0000A16A71B8B177A08FE007908FD00780808
:1026D000FC007708FB00F61C8D2B8314DB3083167F
:1026E000AC000F30AB004930AA007F30A9007E0853
:1026F000B0007D08AF007C08AE007B08AD000A1278
:102700008A15831200200A168A117A08FE007908B9
:10271000FD007808FC007708FB00761C922B7C08F3
:10272000803AFC007B08F7007C08F8007D08F9007F
:102730007E08FA007A08ED007908EC007808EB00D2
:102740007708EA00A7018B1BA7178B136D08831668
:10275000C50083126C088316C40083126B088316AD
:10276000C30083126A088316C200C330C900F53063
:10277000C8004830C7008030C6000A1283125720B4
:102780000A16A71B8B177708EE007808EF00790868
:10279000F0007A08F1008316AC007008AB008312D9
:1027A0006F088316AA0083126E088316A900B00171
:1027B000AF013430AE008630AD000A1283126E27AE
:1027C0000A167A08ED007908EC007808EB00770823
:1027D000EA006A08F7006B08F8006C08F9006D0859
:1027E000FA00F8136D08ED006C08EC007808EB00B7
:1027F0006A08EA00E008031D172CE108031D172CE6
:10280000E31B102CE308031D092C6208003C03188D
:10281000102CED01EC013430EB008530EA00162C71
:10282000ED01EC010730EB008730EA00992CE11B49
:10283000702CE108031D202C6008003C0318702C4C
:10284000E31B492C83108316AC01AB013430AA0082
:102850008630A90083126D088316B00083126C08BD
:102860008316AF0083126B088316AE0083126A08CA
:102870008316AD000A128A15831200200A168A11E7
:102880007A08ED007908EC007808EB007708EA0098
:102890006F2C83148316AC01AB013430AA00863050
:1028A000A90083126D088316B00083126C0883168A
:1028B000AF0083126B088316AE0083126A0883167A
:1028C000AD000A128A15831200200A168A117A08AE
:1028D000ED007908EC007808EB007708EA00992C05
:1028E000E31B992C83148316AC01AB013430AA008E
:1028F0008730A90083126D088316B00083126C081C
:102900008316AF0083126B088316AE0083126A0829
:102910008316AD000A128A15831200200A168A1146
:102920007A08ED007908EC007808EB007708EA00F7
:10293000992C6A08F7006B08F8006C08F9006D081C
:10294000FA008A150A161129E11BBA2C0F30F7007C
:10295000600EF7050A3077020318B12C3030F70704
:10296000B32C6108F7077708ED000A128A153226A2
:102970000A168A110F30E0050A3060020318C22CD3
:102980003030C42CE1136108E0076008ED000A1242
:0E2990008A1532260A168A118A150A162F2B6E
:10300000840183131F308305713083168F000F08EE
:103010008312A81328088316870083128717B40128
:10302000B301B201B101831603170908C039890041
:1030300003131F129F1200300317880083128701A9
:1030400088018901FF300313A800A901AA013030CB
:10305000AB002E30AC003130AD00AE01B501B60191
:103060000930031785000F30F70003138101813009
:10307000840083130008F0390738800064000008DA
:10308000F739F719F03977048000640083160317C5
:103090000908C039890003131F129F12003003175B
:1030A0008800831203131F139F1383169F13831229
:1030B0001F149412A812280883168700831228165A
:1030C0002808831687008312A81128088316870012
:1030D0000130831294000030831694000108C73930
:1030E000283881000F30831290000030F8009200E1
:1030F0000030831692008312281528088316870053
:103100008312970183169B019C0101309D0083125D
:1031100003178701880189010313D001CF010A1227
:103120008A11782A0A168A15D1015108E0000A127C
:103130008A11092B0A168A1583160C1483128B1612
:10314000C0308B0464000A128A11AB2C0A168A154F
:103150000A128A11342D0A168A1581018F018E01F7
:10316000B001AF01B401B301B201B1016400DF01EC
:103170000A128A11E62D0A168A150230E000FA308A
:10318000E5000A128A11F5220A168A15E00BBF28FB
:103190000A128A11EB2E0A168A157A08BA007908E3
:1031A000B9007808B8007708B7000A1246290A164D
:1031B0007A08BE007908BD007808BC007708BB001B
:1031C0000A12202A0A160230E000FA30E5000A123C
:1031D0008A11F5220A168A15E00BE5280A12DD2A63
:1031E0000A167A08C2007908C1007808C00077087A
:1031F000BF000A12852B0A167A08C6007908C50096
:103200007808C4007708C3000A12852C0A167A08C9
:10321000CA007908C9007808C8007708C7008A1171
:1032200000288A157A08CE007908CD007808CC00ED
:103230007708CB002130F700F70B1C292430E4007D
:103240000A128A11D1230A168A152130F700F70BCA
:103250002729B6015230B5004D30ED000A12322652
:103260000A165330ED000A1232260A165430ED00C9
:103270000A1232260A162B30840083130A123F2EBC
:103280000A162030ED000A1232260A16DE015230EC
:103290005E07840083138008031967292130F70033
:1032A000F70B502952305E07840083130008E000BA
:1032B0006008E4000A128A11D1230A168A155E08F2
:1032C000DE0A523E840083130008DF064729B60158
:1032D0005230B500013084005008E1004F08E00092
:1032E0000A12572E0A162030ED000A1232260A164C
:1032F000DE0152305E078400831380080319992988
:103300002130F700F70B822952305E0784008313C7
:103310000008E0006008E4000A128A11D1230A16AE
:103320008A155E08DE0A523E840083130008DF0619
:103330007929B6015230B500053084003A08E3001F
:103340003908E2003808E1003708E0000230E40004
:103350000A1202270A162030ED000A1232260A1637
:10336000DE0152305E078400831380080319D129DF
:103370002130F700F70BBA2952305E07840083131F
:103380000008E0006008E4000A128A11D1230A163E
:103390008A155E08DE0A523E840083130008DF06A9
:1033A000B129B6015230B500063084004208E3006E
:1033B0004108E2004008E1003F08E0000230E4007C
:1033C0000A1202270A162030ED000A1232260A16C7
:1033D000DE0152305E078400831380080319092A36
:1033E0002130F700F70BF22952305E078400831377
:1033F0000008E0006008E4000A128A11D1230A16CE
:103400008A155E08DE0A523E840083130008DF0638
:10341000E929B6015230B500083084003E08E300C7
:103420003D08E2003C08E1003B08E0000230E40017
:103430000A1202270A162030ED000A1232260A1656
:10344000DE0152305E078400831380080319412A8D
:103450002130F700F70B2A2A52305E0784008313CD
:103460000008E0006008E4000A128A11D1230A165D
:103470008A155E08DE0A523E840083130008DF06C8
:10348000212AB6015230B500053084004608E30019
:103490004508E2004408E1004308E0000230E4008F
:1034A0000A1202270A162030ED000A1232260A16E6
:1034B000DE0152305E078400831380080319792AE5
:1034C0002130F700F70B622A52305E078400831325
:1034D0000008E0006008E4000A128A11D1230A16ED
:1034E0008A155E08DE0A523E840083130008DF0658
:1034F000592AB6015230B500053084004A08E3006D
:103500004908E2004808E1004708E0000230E40012
:103510000A1202270A162030ED000A1232260A1675
:10352000DE0152305E078400831380080319B12A3C
:103530002130F700F70B9A2A52305E07840083137C
:103540000008E0006008E4000A128A11D1230A167C
:103550008A155E08DE0A523E840083130008DF06E7
:10356000912AB6015230B500053084004E08E300C0
:103570004D08E2004C08E1004B08E0000230E40096
:103580000A1202270A162030ED000A1232260A1605
:10359000DE0152305E078400831380080319E92A94
:1035A0002130F700F70BD22A52305E0784008313D4
:1035B0000008E0006008E4000A128A11D1230A160C
:1035C0008A155E08DE0A523E840083130008DF0677
:1035D000C92AB6015230B500043084003408E30033
:1035E0003308E2003208E1003108E0000230E40074
:1035F0000A1202270A162030ED000A1232260A1695
:10360000DE0152305E078400831380080319212BEA
:103610002130F700F70B0A2B52305E07840083132A
:103620000008E0006008E4000A128A11D1230A169B
:103630008A155E08DE0A523E840083130008DF0606
:10364000012BB6015230B5002A30ED000A123226A5
:103650000A165F08E0003730E1008A11A42C8A15B1
:103660000D30ED000A1232260A160A30ED000A1259
:1036700032260A16DE0152305E078400831380086A
:103680000319552B2130F700F70B442B5E08DE0A97
:10369000523E840083130008E0006008E4000A1230
:1036A0008A11D1230A168A153B2B2130F700F70B1C
:0E36B000572BCF0A0319D00A6400B728630015
:04400E00FD2CFF3F47
:00000001FF
